:020000020000FC
:1000000008ED04BF03E0009360000091630000FD71
:10001000FCCF08ED04BF00E00093610000E4009312
:10002000E20506EB12E0009368081093690803E00C
:0E0030000093670800EC009366080C94CF0262
:100400000C94CF020C9450020C9450020C945002A5
:100410000C9450020C9450020C9450020C94C102A3
:100420000C9450020C9450020C9450020C94500204
:100430000C9450020C9450020C9450020C945002F4
:100440000C9450020C9450020C9450020C945002E4
:100450000C9450020C9450020C945C020C945002C8
:100460000C9450020C9450020C9450020C945002C4
:100470000C9450020C9450020C9450020C945002B4
:100480000C9450020C9450020C9450020C945002A4
:100490000C9450020C9451020C9450020C94500293
:1004A000189530906008AF93BF93B9E2AD2D3D929F
:1004B000DA2EBF91AF9118952FB60F931F93EF933C
:1004C000FF93309006060FE003211127E1E7F2E0E9
:1004D000E00FF11F0995FF91EF911F910F912FBE32
:1004E00018951FC00EC00DC00CC00BC01AC02DC087
:1004F00008C017C006C005C004C003C002C001C0C8
:1005000035C00091100610911106FAE2E32DEE0FAE
:100510000193119333943092060601E0009308068C
:100520000895E0911006F091110600EC1FEF0E1BEC
:100530001F0BFAE2E32DEE0F0193119333943092E7
:10054000060601E000930806089500911006109138
:100550001106FAE2E32DEE0F0193119333943394D5
:100560003092060601E000930806089500911006F7
:1005700010911106FAE2E32DEE0F01931193E49A24
:10058000089530900B0A30920B0A202E00E0009361
:10059000060601E000930806022DE29A189500E88D
:1005A00001B900ED00B908E00093110400E105B9BC
:1005B0000FE104B908E00093350402E009B902EF45
:1005C00008B908E00093500404E00093700400931D
:1005D00071040093720400937304009374040093F5
:1005E0007504009376040093770404E0009390046C
:1005F00000939104009392040093930403E405BBD9
:1006000003E404BB04E00093B2040093B30400933A
:10061000B4040093B50400E30093A00006E0009347
:10062000010603E6009302060FE7009303060FE0BE
:100630000093050601E000930A0601E0009300061E
:1006400008E01DE30093260A1093270A01E00093B7
:100650000A0A0BE00093000A00E712E000938C0AFC
:1006600010938D0A05E00093800A00E20093C00811
:1006700000E30093C00804E00093C10801E3009385
:10068000C008009101140395D1F40E942810EAE3F8
:10069000F2E2A1E0B4E1159107D0ECE4F2E2A0E4CB
:1006A000B4E110E401D00BC005910D931A95E1F768
:1006B0001DE914BF13E0109300100C94281055246A
:1006C00066247724B5B2C0900C14DD24EE240027F4
:1006D0000CBB0DBB0EBB0FBB00910214037009F0E5
:1006E0008AD4009102140C7009F061D500910214B3
:1006F00005FD0ED5BAD0C6D0CDD024D01ED000E88E
:1007000000936508ECE6F0E274D58BD599D5CDD58C
:100710007894DE100E946804E3990E940209E4992B
:100720000E94300C119B0E947B0A0E94040C0E94C4
:10073000490DE2990E949F0EECCF00910E1406FD28
:10074000499808950F9800EC0E942D100F9A0E946E
:1007500014100F9803E00E942D100EE00E942D103F
:100760000FEF0E942D100F9A007E003881F70F982E
:1007700002E00E942D1008E20E942D1001E00E946C
:100780002D100F9A0F9802E00E942D1009E20E948E
:100790002D100EE80E942D100F9A0F9802E00E9473
:1007A0002D100AE20E942D1000E40E942D100F9AD5
:1007B00050EF48E0309111142091101410E040D017
:1007C0003FEF2FEF14E03CD058EF442710E238D031
:1007D0000F9802E00E942D100BE20E942D1001E004
:1007E0000E942D100F9A0F9802E00E942D100FE02A
:1007F0000E942D1000E00E942D100F9AC8E5DAE249
:1008000050EF48E03091111420911014002718E0A7
:100810005993499339932993099328961A95C1F7C7
:1008200049E04093732A4093802A4AE040938D2AFE
:100830004BE040939A2A48E24093A72AAA240895BD
:100840000F9802E00E942D10012F0E942D10052FFD
:100850000E942D10042F0E942D10032F0E942D1096
:10086000022F0E942D100F9A0895A0E4B4E1E0E059
:10087000FAE220E10D911D910193119312962A95B0
:10088000C9F70895E0E5FAE2002718E001931A9508
:10089000E9F70895A4E0B4E1C0E4DAE244E08D9120
:1008A0009D918C019C0104969695879596958795C8
:1008B00096958795081B190B0993199301969695A0
:1008C0008795280F391F299339934A9541F7089541
:1008D0006D2D6E19653008F40895D9E2CE2D08818A
:1008E000C3950062033651F0043649F0053641F0F5
:1008F000023739F0033731F0E394089504C0C8C0DB
:100900003DC1B1C1D6C1663008F408950881C395D0
:100910000062013699F40881C39500620C3671F4C7
:100920000881C3950062003249F40881C3950062D2
:10093000093631F0063729F00F3621F0E394089597
:1009400002C041C06AC00881C3950D3021F00A3051
:1009500011F0E3940895EC2EC0E0DAE2E0E4F4E173
:100960000E942810F89408811981789400831183DB
:10097000F8940E811F81789404871587F8940A856E
:100980001B857894048B158BF894088919897894C1
:1009900000A311A3F8940A891B89789404A315A3D2
:1009A000F894088D198D789400AB11ABF8940A8DEA
:1009B0001B8D789404AB15AB1DE914BF13E01093A5
:1009C00000100C942810683008F408950881C3952D
:1009D0000F70002E0881C3950B3221F00D3211F0FB
:1009E000E39408951CE2101B112E0881C3950D306D
:1009F00021F00A3011F0E3940895EC2E07E0002175
:100A00001127ECE8F2E2E00FF11F0490A0E4B4E15A
:100A1000A00D0C91010D0C941810683008F4089585
:100A20000881C3950F70002E0881C3950B3221F009
:100A30000D3211F0E39408951CE2101B112E088171
:100A4000C3950B3241F00D3231F00D3049F00A30D0
:100A500039F0E3940895110C6A95683080F7089591
:100A6000EC2E07E00022A0E8B4E1A00D0C91010DEE
:100A70000E9418101124E0E4F5E0E00DF11D099446
:100A80004EC46CC48AC4A8C40895C5C4089508950A
:100A90006C3008F408950881C3950062093639F571
:100AA0000881C3950062033711F50881C395006280
:100AB0000136E9F40881C39500620236C1F4088169
:100AC000C39500620C3699F40881C395006205361F
:100AD00071F40881C3950062003249F40881C3951E
:100AE0000062013631F0033729F0003721F0E3943A
:100AF000089502C016C02AC00881C3950062063757
:100B000059F40881C3950062093631F40881C39510
:100B10000D3021F00A3011F0E3940895EC2E6ED3DD
:100B2000C4C30881C3950062053659F40881C39592
:100B30000062023731F40881C3950D3021F00A308C
:100B400011F0E3940895EC2E59D3AFC30881C395F7
:100B50000062013659F40881C3950062093731F407
:100B60000881C3950D3021F00A3011F0E394089507
:100B7000EC2E0E94AF07E79841D397C36B3008F47F
:100B800008950881C39500620E3611F50881C3955A
:100B900000620136E9F40881C39500620236C1F4AF
:100BA0000881C39500620C3699F40881C3950062F0
:100BB000053671F40881C3950062003249F408815A
:100BC000C3950062013631F0033729F0003721F078
:100BD000E394089502C016C02AC00881C39500623C
:100BE000063759F40881C3950062093631F408814B
:100BF000C3950D3021F00A3011F0E3940895EC2EE6
:100C0000FDD253C30881C3950062053659F40881AB
:100C1000C3950062023731F40881C3950D3021F08D
:100C20000A3011F0E3940895EC2EE8D23EC3088117
:100C3000C3950062013659F40881C39500620937F3
:100C400031F40881C3950D3021F00A3011F0E3949E
:100C50000895EC2E00910E1407FDE79A07FF0E94FD
:100C6000AC07CCD222C3663008F408950881C3953E
:100C700000620536A9F40881C3950062033781F448
:100C80000881C3950062053659F40881C395006256
:100C9000043731F40881C3950D3021F00A3011F08A
:100CA000E3940895EC2E08ED04BF01E000934100A9
:100CB00008950881C3950062053621F0083619F0C1
:100CC000E394089501C07AC26B3008F40895088156
:100CD000C3950062043771F40881C3950062003245
:100CE00049F40881C3950062003731F0033769F099
:100CF0000637A1F0E39408950881C3950062003798
:100D0000D1F00337C9F0E39408950881C3950062D8
:100D1000003399F00E3691F0E39408950881C3955D
:100D20000062013661F0023659F0003751F00337A6
:100D300049F0E394089507C039C05CC0ACC012C14B
:100D400061C19DC1EBC16C3008F408950881C39561
:100D500000620D33E9F40881C3950F70002E0AE09C
:100D6000009E0881C3950F70000E0AE0009E088166
:100D7000C39500620E3261F40881C3950F7011278C
:100D8000000E111E0881C3950D3021F00A3011F0BC
:100D9000E3940895EC2E002D112009F00027ACE01B
:100DA0000E941810C0900C1429D24AC20881C39521
:100DB00000620D33B1F40881C3950F70002E0AE074
:100DC000009E0881C3950F70000E0AE0009E088106
:100DD000C3950F70000E0881C3950D3021F00A30C5
:100DE00011F0E3940895EC2EADE0002D0E94181050
:100DF00005D226C20881C39500620D33B1F4088183
:100E0000C3950F70002E0AE0009E0881C3950F70F5
:100E1000000E0AE0009E0881C3950F70000E088145
:100E2000C3950D3021F00A3011F0E3940895EC2EB3
:100E3000AEE0002D0E94181005FF0ED006FD499867
:100E400006FF499AE79B05C007FD03C00E94AC0757
:100E5000E798D4D1F5D129C20F9300E20093E305BE
:100E60000DE20093A60801E00093A30801E00093BF
:100E7000A50800E00093A70836D346F006E00093EB
:100E8000A80831D31EF003E00093A40800270093C4
:100E9000A3080F9108956D3008F408950881C39553
:100EA00000620D33B1F50881C3950F70002E0AE082
:100EB000009E0881C3950F70000E0AE0009E088115
:100EC000C3950F701127000E111E8001000C111C1C
:100ED000000C111C000E111E000C111C0881C39582
:100EE0000F701127000E111E8001000C111C000C48
:100EF000111C000E111E000C111C0881C3950F70EF
:100F00001127000E111E0881C3950D3021F00A3003
:100F100011F0E3940895EC2E8091FE149091FF144B
:100F2000019621F0C001019609F00895AEEF002D61
:100F30000E941810AFEF012D0E9418105FD171C1EF
:100F40006894B0F80895E894B0F808956894B1F8FA
:100F50000895E894B1F808956894B6F80895E8946F
:100F6000B6F808956C3008F408950881C3950062BE
:100F70000D33E9F40881C3950F70002E0AE0009E3E
:100F80000881C3950F70000E0AE0009E0881C3958A
:100F900000620E3261F40881C3950F701127000EB4
:100FA000111E0881C3950D3021F00A3011F0E39431
:100FB0000895EC2E08E710E00016110630F008E165
:100FC00011E00015110508F08001209104140213AE
:100FD00002D014D135C10F93009102140360A2E036
:100FE0000E9418100F91A4E00E941810012FA5E094
:100FF0000E9418104FDCE09AA8980E9414108FD11C
:10100000ADD108956C3008F408950881C39500624D
:101010000D33E9F40881C3950F70002E0AE0009E9D
:101020000881C3950F70000E0AE0009E0881C395E9
:1010300000620E3261F40881C3950F701127000E13
:10104000111E0881C3950D3021F00A3011F0E39490
:101050000895EC2E00EF10E00016110630F006E2C5
:1010600012E00015110508F08001AAE00E94181096
:10107000012FABE00E9418100DDCC0D0E1C06C3035
:1010800008F408950881C39500620D33E9F40881DE
:10109000C3950F70002E0AE0009E0881C3950F7063
:1010A000000E0AE0009E0881C39500620E3261F4D2
:1010B0000881C3950F701127000E111E0881C3957A
:1010C0000D3021F00A3011F0E3940895EC2E08E77A
:1010D00010E00016110630F008E111E000151105CE
:1010E00008F0800120910814021302D087D0A8C014
:1010F0000F93009102140062A2E00E9418100F9159
:10110000A8E00E941810012FA9E00E941810C2DB6D
:10111000E69AAE980E9414107ED108956C3008F4BF
:1011200008950881C39500620D33E9F40881C395E1
:101130000F70002E0AE0009E0881C3950F70000E0C
:101140000AE0009E0881C39500620E3261F40881B6
:10115000C3950F701127000E111E0881C3950D3025
:1011600021F00A3011F0E3940895EC2E0CE310E026
:101170000016110630F008E111E00015110508F025
:10118000800120910614021302D038D059C00F9369
:10119000009102140C60A2E00E9418100F91A6E0CA
:1011A0000E941810012FA7E00E94181073DBE19A2B
:1011B000A9980E941410F1D00FD108950881C39509
:1011C00000620F3659F40881C3950062073731F485
:1011D0000881C3950D3021F00A3011F0E394089591
:1011E000EC2E0CD02DD061C0059109930023E1F7BE
:1011F0000895D8E2C0E0F8DFFF24E39AE39B089566
:1012000001D0FCCFD8E2CF2D0991002311F4E3984F
:1012100008951091640815FF089500936208FC2E4C
:101220000895F1E2E4EAD8E2C0E0DEDFF8E22091DE
:10123000FE143091FF14EFE058D0FF24E39ADECF84
:10124000F1E2ECEBD8E2C0E0CFDFF8E22091041449
:1012500030910514EBE14FD05ED02091061430910F
:101260000714E5E248D057D02091081430910914B2
:10127000EFE241D050D020910A1430910B14E9E3F1
:101280003AD049D020910C143327E3E434D043D032
:1012900020910D143327EDE42ED020910E14332726
:1012A000E5E529D0FF24E39AA9CFF2E2E8E1D8E20C
:1012B000C0E09ADFF8E2E6E1B6FC06D0E6E1E799A5
:1012C00003D0FF24E39A9ACF25E421932EE62193BD
:1012D00021E6219322E621932CE6219325E6219312
:1012E00024E6219320E22193089517E200E109D03A
:1012F00013E008EE06D0112704E603D00AE001D07F
:1013000001E040E34395201B310BE0F7200F311F34
:101310004A954193089540834EE242930895009187
:1013200004141EE1101B06E1109F00918014112788
:1013300007FD1095001A110A90013F70306948E5C9
:1013400000E288D085D60091021400F900930214BF
:101350001DE914BF11E0109300107AC60091041427
:101360001EE1101B06E1109F00918114112707FD5B
:101370001095001A110A90013F70306948E500E1AC
:1013800069D066D60091021401F9009302141DE998
:1013900014BF11E0109300105BC6009106141CE20C
:1013A000101B00E1109F00918214112707FD10957A
:1013B000001A110A90013F7030694AE500E24AD0F4
:1013C00047D60091021402F9009302141DE914BFDC
:1013D00011E0109300103CC6009106141CE2101B93
:1013E00000E1109F00918314112707FD1095001A4A
:1013F000110A90013F7030694AE500E12BD028D6F0
:101400000091021403F9009302141DE914BF11E0C6
:10141000109300101DC6009108141EE1101B06E178
:10142000109F00918514112707FD1095001A110ACD
:1014300090013F7030694CE500E10CD009D6009175
:10144000021405F9009302141DE914BF11E0109372
:101450000010FEC50093E3050DE20093A60801E02D
:101460000093A30801E00093A50801EC0093A708EE
:1014700032D06EF11091A80802E00093A4082BD09E
:1014800036F10091A80802E00093A40824D0FEF0F1
:101490000091A80817FD04C002E00093A408E8CF5B
:1014A00007E00093A40800EC0093A7081CD07EF08E
:1014B0004093A80818D05EF03093A80814D03EF0EE
:1014C0002093A80810D01EF003E00093A408002782
:1014D0000093A30808959BD50091A50807FD0895E2
:1014E0009FD5D6F7089593D50091A50806FD0895D8
:1014F00097D5D6F708950F9800E90E942D100E9405
:101500002D10502F0E942D10402F0E942D10302F93
:101510000E942D10202F0E942D10102F0E942D10A0
:10152000102E0E942D10002E0F9A43FF0895CA011D
:10153000042F5695479546954695552703704C7F41
:10154000402B1F7059F0123021F008F00895012C43
:101550001124E3EBFAE0E40FF51F0994ECE0FBE063
:10156000E40FF51F099408950895089508950895C6
:101570000895089508950895089508950895089583
:101580000895089530C016CDF1CDA1CD63CD03CC23
:101590002BCC089508954CCC0895089526C0089545
:1015A00008950895089535C00895089508950895FB
:1015B0000895089508950895089508950895089543
:1015C000089508950895A8CC08950895089508955C
:1015D0000895089508950895089508950895089523
:1015E0000895089508950DBA0895A0E1002D0E9470
:1015F0001810A1E1012D0E9418100F9802E00E941E
:101600002D100FE00E942D1000E80E942D100F9A5F
:101610009EC806FEAECA1ECB3FC040C041C042C0FD
:1016200043C008950895089508950895089508956C
:101630000895089508953AC03CC04BC05AC069C08F
:1016400078C083C0089508958CC00895089595C00A
:101650000895089508950895A0C0089508950895DF
:101660000895089520CB0895089508950895089544
:1016700008950895089508959DC0ACC008950895F3
:101680000895089508950895089508950895089572
:101690000895089508950895E89A0895E99A089597
:1016A000EA9A0895EB9A0895EC9A08950FE10DBB1C
:1016B000089572E060910514509104149093B32A38
:1016C0008093B42A7093B72A6093B82A5093B92AAA
:1016D000089572E060910714509106149093B32A14
:1016E0008093B42A7093B72A6093B82A5093B92A8A
:1016F000089572E060910914509108149093B32AF0
:101700008093B42A7093B72A6093B82A5093B92A69
:10171000089572E060910B1450910A149093B32ACB
:101720008093B42A7093B72A6093B82A5093B92A49
:10173000089571E060910C149093B32A8093B42AB9
:101740007093B72A6093B82A089571E060910D14E0
:101750009093B32A8093B42A7093B72A6093B82ADF
:10176000089571E060910E149093B32A8093B42A87
:101770007093B72A6093B82A089572E060911114AB
:10178000509110149093B32A8093B42A7093B72A7F
:101790006093B82A5093B92A089571E06B2DE799A8
:1017A00060649093B32A8093B42A7093B72A6093AD
:1017B000B82A089572E06091FF145091FE1490933E
:1017C000B32A8093B42A7093B72A6093B82A5093AF
:1017D000B92A089576E061E054E04FE137E027E070
:1017E00014EE9093B32A8093B42A7093B72A60932F
:1017F000B82A5093B92A4093BA2A3093BB2A20932F
:10180000BC2A1093BD2A08950DE0A09EC8E5DAE237
:10181000C00DD11D1C811F70F9F0FE011930D0F4EC
:101820000F9800EA0E942D100E942D100F9A02FDC1
:1018300008950F9800E40E942D101B5F09910E94EB
:101840002D101A95D9F70F9A00000F9801E80E9401
:101850002D100F9A11271483A394A3FCAA24089592
:10186000E498A0E0BAE2C0E2DAE2E0E4F4E16FE09A
:101870002AD06A95E9F747D0C0E2DAE2E0E5FAE279
:101880000E811F8124813581468157810024200FDC
:10189000311F401D501D24833583468357830881A3
:1018A000198120813181428153810024200F311F11
:1018B000401D501D2083318342835383E0E4FAE2CC
:1018C0004BD0A1D00895F8940D911D917894219159
:1018D0003191021B130B10F40027112730E82191DE
:1018E000129FA001029F0027300D411D501F10E8DC
:1018F0000191509F9001409F4427100D211D341FDE
:10190000299339930895E894F8940D911D91789452
:1019100021913191021B130B28F46894015010405F
:101920000095109530E82191129FA001029F002799
:10193000300D411D501F10E80191509F9001409FB4
:101940004427100D211D341F26F4209530952F5F5C
:101950003F4F29933993089500270FBB0E891F89A4
:10196000208131810217130730F022813381201743
:10197000310708F0F89A0C851D85248135810217FE
:10198000130730F0268137812017310708F0F99AC4
:101990000C891D89208531850217130730F02285B7
:1019A00033852017310708F0FA9A0C811D812485B0
:1019B00035850217130730F0268537852017310744
:1019C00008F0FB9A088D198D22E330E020173107CB
:1019D00008F0FC9A088919892AEF30E020173107AE
:1019E00008F0FD9A0A891B8924EB30E020173107A3
:1019F00008F0FE9A0E811F812AEF30E02017310790
:101A000008F0FF9A089500270EBB0C8D1D8D2081D4
:101A100031810217130730F02281338120173107FB
:101A200008F0F09A0885198524813581021713077B
:101A300030F0268137812017310708F0F19A0A81AA
:101A40001B81248535850217130730F026853785DD
:101A50002017310708F0F39A0A8D1B8D22E330E03E
:101A60002017310708F0F49A0A851B852AEF30E029
:101A70002017310708F0F59A088119812AEF30E024
:101A80002017310708F0F79AFA99F29AFE99F69A18
:101A900008950DB30F7109F40895D8E2C0E0E899F4
:101AA0000ED0E99967D0EA99C0D0EB9904D1EC99AE
:101AB0000DD1AA24FF24E39A00270DBB0895FC2E24
:101AC000F0E2ECEB91DBBAE2ACE508E00D9320919B
:101AD0003C2A30913D2A3D932D93F8E2E4E0EF0D4E
:101AE0000ADC19DC2091362A3091372A3D932D9358
:101AF000F8E2EFE0EF0DFFDB0EDC2091282A3091B9
:101B0000292A3D932D93F8E2EAE1EF0DF4DB03DCA3
:101B100020912C2A30912D2A3D932D93F8E2E5E275
:101B2000EF0DE9DBF8DBBAE2A9E606E00D932091C0
:101B3000342A3091352A3D932D93F8E2EFE2EF0DF0
:101B4000DADBE9DB2091222A3091232A3D932D9381
:101B5000F8E2EAE3EF0DCFDBDEDB2091242A3091BF
:101B6000252A3D932D93F8E2E5E4EF0DC4DBD3DBAA
:101B7000CA950895FC2EF1E2EAE036DBBAE2A6E768
:101B800008E00D9320913A2A30913B2A3D932D9302
:101B9000F8E2E4E0EF0DAFDBBEDB2091382A3091B4
:101BA000392A3D932D93F8E2EFE0EF0DA4DBB3DB90
:101BB00020912A2A30912B2A3D932D93F8E2EAE1D5
:101BC000EF0D99DBA8DB2091302A3091312A3D932B
:101BD0002D93F8E2E5E2EF0D8EDB9DDBBAE2A3E8A0
:101BE00006E00D932091322A3091332A3D932D93B4
:101BF000F8E2EFE2EF0D7FDB8EDB2091202A3091BF
:101C0000212A3D932D93F8E2EAE3EF0D74DB83DBA9
:101C10002091262A3091272A3D932D93F8E2E5E47E
:101C2000EF0D69DB78DBCA950895FC2EF1E2E8E55B
:101C3000DBDABAE2A0E904E00D9356EB6091502A9A
:101C4000659F80016091522A659F90016091532A9F
:101C5000659F402D6091512A659F100D211D341FF5
:101C6000442750E8150F241F341F3D932D93F8E2AD
:101C7000E5E0EF0D3ADB56EB6091542A659F800159
:101C80006091562A659F90016091572A659F402D6B
:101C90006091552A659F100D211D341F442750E87F
:101CA000150F241F341F3D932D93F8E2E4E1EF0D4F
:101CB0001CDBCA950895FC2EF1E2E8E795DABAE25A
:101CC000ADE901E00D9328D0CA950895FC2EF1E20C
:101CD000E2E88ADABAE2AAEA04E00D932CB33327E9
:101CE0002D93F8E2E3E0EF0D06DB2DB333272D93C0
:101CF000F8E2EBE0EF0DFFDA2EB333272D93F8E295
:101D0000E3E1EF0DF8DA2FB333272D93F8E2EBE19F
:101D1000EF0DF1DACA95089520913E2A30913F2ABD
:101D20002D934BE237FD05D0F8E2E2E0EF0D419351
:101D3000E2CA4DE221503040209530950895E29856
:101D400043940CD032D046D04FD0EBD016D1E0998E
:101D50002CD1E1993DD1E6994ED108950EB31FB330
:101D6000012B102F1295012B5A946A947A9415E046
:101D700000FF510E01FF610E02FF710E57FC5394DC
:101D800067FC639477FC739418E2511618F0512E97
:101D9000E09AA898611618F0612EE19AA998711638
:101DA00018F0712EE69AAE9808951EB342FE1FB346
:101DB000012F129501231FE00123009326040295B1
:101DC0000093450402950127009325040295009392
:101DD00046040895CA9409F00895C0900C14009127
:101DE0000D140F710DBB089500910E1405FF089599
:101DF00040FE089541FE089542FE08954427C0E242
:101E0000DAE2A89905D0A99911D04423E9F40895FC
:101E10008A8D9B8D088D198D801B910B04961AF06D
:101E2000099712F408954260416008958A859B8560
:101E300008891989801B910B0A961AF0459712F4AC
:101E4000089548604460089500E20093E3050DE2C0
:101E50000093A60801E00093A30801E00093A50801
:101E600001EC0093A7081CE0C0ECDAE234DB86F05A
:101E70000091A80809931A9521F002E00093A408A4
:101E8000F5CF07E00093A4080091C92A07FD04C01C
:101E900000270093A3080895C0ECDAE2E89440FF1D
:101EA00011C08A8199811D81181B119541FD04C0C3
:101EB000163144F4019603C01B3E24F001978A8337
:101EC0009983689442FF11C088859F811B85181BE8
:101ED000119543FD04C0103244F4019603C0113E35
:101EE00024F0019788879F836894BEF400E40883F8
:101EF00002E40B831F8108851C830D8300EC009393
:101F0000A70817E0F0DA4EF01A9521F00991009336
:101F1000A808F8CF03E00093A40800270093A308C3
:101F2000089500910E1407FF089580914C2A909116
:101F30004D2A44960091222A1091232A0817190746
:101F4000B0F42091242A3091252A2817390778F4F3
:101F500044970817190708F008952817390708F05B
:101F60000895B6FE08950E94AF07E79A0895E79B8B
:101F700008950E94AC07E798089505B30B251CB39C
:101F80001095012300FD05C001FD07C006FD09C035
:101F9000089501E00093A704089502E00093A704C8
:101FA000089500E40093A7040895002750120895AF
:101FB00080913C2A90913D2AC29708F00895809123
:101FC000362A9091372AC29708F00895E09808952C
:101FD0000027601208958091282A9091292AC2979B
:101FE00008F0089580912C2A90912D2AC29708F02C
:101FF0000895E19808950027701208958091342A79
:102000009091352AC29708F00895E6980895002720
:1020100000938A0A00938B0A01E00093860A0895D0
:102020000091860A00FB0895F2DFFADFF6F70895C3
:102030001F93BF93B4E11C91101303D0BF911F9164
:10204000089506D00C931DE914BF13E010930010FF
:102050001091021011FDFCCF08950093C408009167
:10206000C30807FFFCCF0091C40808950D0A4D690D
:102070006C6C73776F6F6420456E67696E6565720F
:10208000696E67203930305720506F776572204471
:102090006973747269627574696F6E20556E6974C4
:1020A0000D0A4669726D7761726520766572736993
:1020B0006F6E3A20312E30340D0A00005661613DBA
:1020C0002A2A2E2A5620205661623D2A2A2E2A5676
:1020D00020205673613D2A2A2E2A562020567362EC
:1020E0003D2A2A2E2A56202056703D2A2A2E2A566C
:1020F00020205662613D2A2A2E2A562020566262EE
:102100003D2A2A2E2A560D0A00004961613D2A2ADD
:102110002E2A4120204961623D2A2A2E2A41202070
:102120004973613D2A2A2E2A4120204973623D2AA3
:102130002A2E2A41202049703D2A2A2E2A41202079
:102140004962613D2A2A2E2A4120204962623D2AA5
:102150002A2E2A410D0A00004562613D2D2A2A2AB5
:102160002A2A6D414820204562623D2D2A2A2A2ACA
:102170002A6D41480D0A0000543D2B2A2A2A430D9E
:102180000A0052303D2A2A2A202052313D2A2A2A8A
:10219000202052323D2A2A2A202052333D2A2A2A40
:1021A0000D0A000053657269616C206E756D626581
:1021B000723A202A2A2A2A2A0D0A0000436F6E66E4
:1021C000696775726174696F6E2073657474696E86
:1021D00067733A2056613D2A2A2E2A5620205673CC
:1021E0003D2A2A2E2A56202056703D2A2A2E2A566B
:1021F000202056623D2A2A2E2A56202050703D2A41
:102200002A2E2A53202050733D2A2A2A2020533078
:102210003D2A2A2A0D0A0000456E61626C65642021
:1022200066656174757265733A205061793A4469E4
:102230007361626C65640D0A00001100FFFFB40059
:10224000B400B400A4010AFF00FF0100E07FC20453
:102250000000CB030000CB03E07FC2040000980223
:10226000E07FC2040000980200000000E07FC2048A
:10227000E07FC20400009802000098024074A801A8
:102280004074A80100009802001FA9013A2E121AFA
:042290002A2A060AE6
:00000001FF
